:020000020000FC
:100000000C942E000C942E000C946A100C94AD10DD
:100010000C942E000C94E4100C942E000C942E00E2
:100020000C942E000C942E000C9438100C942E007E
:100030000C942E000C942E000C942E000C942E0088
:100040000C942E000C942E000C942E000C942E0078
:100050000C942E000C942E000C94BA10F89404E02A
:100060000EBF0FEF0DBF222402E01DEF04B915B93A
:1000700004E218E30DB91EB900E010EF00BB11BB9C
:100080000FE000937E000EE000936400B1E0A0E07A
:100090002D92B430E9F707EB0093E50003E00093FD
:1000A000E6000EEE0093E70008EC0093E40063E046
:1000B00001E400937C0003E100937A0007E00093E1
:1000C0007E0001EF00936C0003E000936B0000ECF6
:1000D0000DBB09E004BD00E007BD03E00093B000E4
:1000E00001E00093700008E00093B600772404E07C
:1000F000009322010FEF0093170108EC00932301F6
:10010000209224017598F8D0DDD010D1789419D1BF
:1001100094D6F3990E945411F39BE8D3F39B45D4F2
:10012000F39B0E94B408F39B16D0F39B70D0F39B13
:1001300026D167D70E947111C8D4603021F403B171
:1001400001780C6705B907E003BF88952F9A289AB4
:1001500006E003BFDDCF0AB501FD0895F6990895C5
:100160000BB502FD0CC000911801003009F0089594
:1001700000911901DAD100E3C01609F00895A7E64D
:10018000B1E000911E0189E0089FA00DB11D109102
:100190001A0100911901EBD10D910F3F19F0C01612
:1001A00008F051E00D910F3F19F0C01608F052E031
:1001B0000D910F3F19F0C01608F051E00D910F3F5F
:1001C00019F0C01608F052E00D910F3F19F0C0165B
:1001D00008F051E00D910F3F19F0C01608F052E001
:1001E0000D910F3F19F0C01608F051E00D910F3F2F
:1001F00019F0C01608F052E00D910F3F19F0C0162B
:1002000008F053E00BB502600B7F0BBD08950BB5F2
:1002100001FF08950D7F0BBD503031F0513041F09A
:100220005230B9F0533031F132D53CD546D508952E
:1002300039D543D54DD5C0903701D09038012BD05A
:1002400000912301109124010C151D0519F161D5B0
:1002500021C01DD532D547D5C0903901D0903A0183
:100260001AD000912301109124010C151D0591F065
:100270005BD510C017D50BD541D5C0903B01D090B0
:100280003C0109D000912301109124010C151D059A
:1002900009F055D508950091350150933501501757
:1002A00009F40895C0922301D09224010895A9E190
:1002B000B1E010EE81E095E00D9173D113959A9520
:1002C000D9F70895A9E1B1E010EE81E095E060D1A1
:1002D0000D9313959A95D9F70895A7E6B1E010E02C
:1002E00080E09AE5CD9054D1C01611F00C2D59D173
:1002F00013959A95B9F70895A7E6B1E010E080E06C
:100300009AE546D10D9313959A95D9F70895A7E3E9
:10031000B1E01AE580E096E0CD903AD1C01611F038
:100320000C2D3FD113959A95B9F70895A7E3B1E045
:100330001AE580E096E02CD10D9313959A95D9F7A4
:10034000089504E607BD0FEF00932A0120922901CA
:1003500005B3026005BB00916E00026000936E0061
:1003600000916E0001FDFCCF0FEF0093150120926C
:100370000E0120920F0120921301F39A08950AB5FD
:1003800004FF0895839A8B9A03E400937C00000095
:100390000000000004EC00937A0000917A0006FD52
:1003A000FCCF009178001091790000932001109308
:1003B000210101E400937C0000000000000004EC37
:1003C00000937A0000917A0006FDFCCFF8940AB5FC
:1003D0000F7E0ABD789483988B9804E000937A008E
:1003E00000917800109179000093060110930701A5
:1003F00080EE882E8EE2982E80912001909121012E
:10040000801B910B199D7001089D6001189DD00CF7
:10041000E11CF21C909ED00CE11CF21C21E0002794
:100420001127C81AD90AE208F20818F0020F121DA3
:10043000F8CFF4E2EAEA8591959132978017910717
:1004400018F4CC24DD242FC022E38EECC82E8FEFCD
:10045000D82E859195918030920541F080179107B3
:1004600048F0E82EF92EC20ED21CF3CF0FEFC02EAB
:10047000D02E19C0EF92FF92E81AF90A81E0882E77
:1004800088279927E21AF20818F0880D921DFACFF2
:1004900021E0FF90EF90E81AF90AE016F1061CF04F
:1004A000C20ED21CF8CFC0920001D0920101F39B82
:1004B00082D00BB501600BBD0E942A110895102F48
:1004C000107F1295D12E10E3D10E1AE3D11610F041
:1004D00017E0D10E102F1F70C12E10E3C10E1AE3CA
:1004E000C11610F017E0C10E0895CC24DD24EE24CF
:1004F000FF24083E83E0180720F0085E1340F394C1
:10050000F8CF043680E0180720F004561040E3943A
:10051000F8CF0A3018F00A50D394FBCFC02E00E376
:10052000F00EE00ED00EC00E0895CC24DD24EE2493
:10053000043618F00456E394FBCF0A3018F00A5042
:10054000D394FBCFC02E00E3E00ED00EC00E089572
:10055000EE24DD24CC240C3318F00C53E394FBCFB1
:10056000063018F00650D394FBCFC02EECCF86E0B7
:10057000189FC02C0A3018F00A50C394FBCF08957E
:10058000CC24063018F00650C394FBCF0C2D0895F0
:10059000F999FECFF89482BD11BDF89A00B5789410
:1005A0000895F999FECFF89482BD11BD00BDFA9A65
:1005B000F99A789408950091000110910101C0907A
:1005C0000201D09003010093020110930301E09017
:1005D0000401E09205010C191D090093040180E05B
:1005E00019F082E00AF081E00E0D0AF40195003066
:1005F00009F40395C02E04E0C01608F0C02E009147
:10060000000110910101D0902301E09024010D1907
:100610001E096AF094E10F301205C0F498E006302C
:100620001205A0F494E00230120580F40EC010957B
:10063000019598E10F30120548F490E1063012055B
:1006400028F49CE00230120508F490E0980F909393
:100650003201EEE2F3E0E90FF21D09941BC01DC068
:100660001FC021C021C023C026C01DC028C029C072
:100670002CC019C02DC02EC031C015C033C034C02D
:1006800036C011C038C03AC03CC00DC03DC03FC0EC
:1006900041C009C0209227010895209227010895A2
:1006A000209227010895089583E037C008958AE0D5
:1006B0008C9D802D32C08AE08C9D802D48C08AE0C0
:1006C0002CC084E18C9D802D28C0209227010895A4
:1006D00083E03DC08AE08C9D802D1FC08AE08C9D08
:1006E000802D35C08AE033C020922701089584E12F
:1006F0008C9D802D2CC082E310C0089584E60DC02F
:10070000089582E30AC0089582E321C0089582E338
:100710001EC0089584E61BC008950BB503FD1AC0E2
:100720002092270100910E0110910F01081B120960
:1007300000930E0110930F0120F420920E012092DD
:100740000F010091120106FD0895F19A27C00BB523
:1007500003FDE6CF2092270100910E0110910F01B9
:10076000080F121D00930E0110930F01C09010018D
:10077000D0901101C01AD10A62F4009110011091B9
:10078000110100930E0110930F01C1948C1908F40C
:1007900008950091120107FD0895F19880932701B3
:1007A000F2990895F09A00911201007C00931201D1
:1007B00080930C0120920D0108951AB511FF08D203
:1007C00011FFE5D111FDEED111FDF7D108956AD0E9
:1007D000A7E6B1E000911E0189E0089FA00DB11DC0
:1007E000A0933001B093310184E090E00D91C8DE18
:1007F000091721F093959831C9F0FACF0E9111960F
:100800001C910117B0F4092F006810E36FD10D910E
:100810000A95B6DE0395091749F00F93092F006872
:1008200010E364D10F9193959831A9F78A95E9F671
:1008300008951196FBCF0C910F9334D084E0A091D2
:100840003001B091310190E00D919ADE091721F04D
:1008500093959831C9F0FACF0E9111961C9101171A
:10086000F8F4092F006810E341D10D910A9588DE54
:100870000395091749F00F93092F006810E336D14B
:100880000F9193959831A9F78A95E9F60F9178DE43
:100890000F9310E22BD10F91006810E127D108953A
:1008A0001196F2CF209240012092540120924501EE
:1008B0002092590100914A01007800934A01009169
:1008C0005E01007800935E0100914F010F7B009361
:1008D0004F01009163010F7B009363010895AFE323
:1008E000B1E018E22D921A95E9F70895F699089566
:1008F00000911F01002341F1053009F055C000911E
:10090000230110912401F1DD0E2D003309F40FE3D2
:1009100010E17CD00D2D7AD00C2D78D000E476D06B
:100920000FE310E273D00FE371D00FE36FD00FE34A
:100930006DD0009146010F770093460100915A0156
:100940000F7700935A011CC000912E01002361F51E
:10095000009128010770003091F2013029F50091D3
:10096000000110910101C1DD0E2D003309F40FE3E8
:1009700010E34CD00D2D4AD00C2D48D000E446D0C9
:1009800000914F010F7700934F01009163010F77A2
:1009900000936301009146010068009346010091B5
:1009A0005A01006800935A010895F699089500913C
:1009B0001F01003051F500912E01002331F5009107
:1009C00028010770043009F5009146010F77009364
:1009D000460100915A010F7700935A0100911A01C4
:1009E000A4DD0D2D003309F40FE310E30FD00C2D1F
:1009F0000DD00091190199DD0D2D08D00C2D06D0D8
:100A000000914F01006800934F0108950053CF9269
:100A1000DF92EF93FF93AF93BF931F93912F107FBC
:100A20001295113029F0123039F0133049F012C00C
:100A3000AFE3B1E018D00EC0A3E5B1E014D00AC016
:100A4000AFE3B1E00F939F930ED0A3E5B1E09F9188
:100A50000F9109D01F911395BF91AF91FF91EF9125
:100A6000DF90CF900895FDE0E8EB82E0089FE00D75
:100A7000F11DD590C490FDE0E0E88EE09F70989F56
:100A8000E00DF11D9EE0C0FAD694C7941591012F98
:100A9000187F169516951695AF93BF93A10FB21DAB
:100AA0008C91102F177001E0103019F0000F1A957B
:100AB000FBCF26F0009580238C9302C0802B8C9373
:100AC000BF91AF919A95F9F6089514E100912E0126
:100AD00001FD03C0AFE3B1E002C0A3E5B1E0CCEE9D
:100AE000D0E00D9109931A95E1F70895EF93FF93E4
:100AF000EEE0FEE009C0EF93FF93FEE0E6E204C003
:100B0000EF93FF93EEE2FEE0AF93BF931F938F93BB
:100B1000107F1295113029F0123039F0133049F05E
:100B200012C0AFE3B1E016D00EC0A3E5B1E012D021
:100B30000AC0AFE3B1E00F93EF93FF930BD0FF91A7
:100B4000EF910F91F2CF8F911F91BF91AF91FF91D4
:100B5000EF91089507FB0F71E00FF21D1591012F22
:100B6000187F169516951695A10FB21D8C91102F12
:100B7000177001E0103019F0000F1A95FBCF26F026
:100B8000009580238C930895802B8C930895009179
:100B9000490101600093490100915D0101600093EA
:100BA0005D010895009149010E7F00934901009174
:100BB0005D010E7F00935D01089500914E0101607B
:100BC00000934E010091620101600093620108955B
:100BD00000914E010E7F00934E01009162010E7F45
:100BE00000936201089500914F01006800934F0146
:100BF00000916301006800936301089500914F0123
:100C00000F7700934F01009163010F770093630109
:100C100008950091460100680093460100915A0131
:100C2000006800935A010895009146010F770093E0
:100C3000460100915A010F7700935A0108950091DF
:100C40004F01109163010F73107C102B10936301FF
:100C500000914A0110915E0100781F77102B1093CC
:100C60005E01089580914F01807C80934F018091B7
:100C70006301807C8093630180914A018F77809328
:100C80004A0180915E018F7780935E010895009103
:100C900042010E7F00934201009156010E7F0093A6
:100CA00056010895009147010E7F0093470100917E
:100CB0005B010E7F00935B01089500914C010E7F54
:100CC00000934C01009160010E7F00936001089534
:100CD00000914201016000934201009156010160C0
:100CE0000093560108950091470101600093470168
:100CF00000915B01016000935B01089500914C013C
:100D0000016000934C01009160010160009360015B
:100D10000895009142010E7F009342010091560117
:100D20000160009356010895009147010E7F0093E2
:100D3000470100915B01016000935B010895009100
:100D40004C010E7F00934C01009160010160009303
:100D50006001089500913F01016000933F010091FF
:100D60005301016000935301089500913F010E7FEC
:100D700000933F01009153010E7F009353010895AA
:100D80007E7C2C05077F2F5557567D2D2E067B79AF
:100D9000010204542B5153527A292A03898B3B12A6
:100DA0001088386260618A3A39118C8E1615136387
:100DB0003C6664658D3E3D14243F040600DB008FD5
:100DC00000E600ED00FD140100FF00EF00C022006E
:100DD0000C0000C81100000000E300F7128F00397A
:100DE000120F0079007100BD00F61209001E0C7090
:100DF000003805360936003F00F3083F08F300EDE0
:100E00001201003E243028362D00150024095830E8
:100E1000080931595A320A0B335B5C340C0D355DCD
:100E2000865E360E0F378081828384855F00005096
:100E300078281718406890678F00F39B0895F19BFE
:100E400037C000910C0110910D010E3A81E0180796
:100E500071F4809114018093150180914A018160A1
:100E600080934A0180915E01816080935E01809150
:100E7000140190911501891B08F488278A30C0F06D
:100E80000091450100FD0EC020920E0120920F013D
:100E900000914501016000934501009159010160F5
:100EA0000093590100E110E000930C0110930D0133
:100EB000F299089510911301103041F0123019F198
:100EC0001430E1F1163009F008955CC0F198F09A01
:100ED000209212011395109313010CE310E196DD9B
:100EE0000FE394DD0CE392DD0FE390DD0FE310E2FE
:100EF0008DDD0CE38BDD0FE389DD0CE387DD00E1A5
:100F000000930D0108950AB502FD26C0F49B0895D3
:100F1000F498009108010430D1F704E00093130124
:100F200001E410E373DD04E471DD01E46FDD00E54D
:100F30006DDD20920E0120920F010895F19AF09A32
:100F40002092120113951093130102EC11E000930B
:100F50000C0110930D01089504E00093130104E4C3
:100F600010E354DD05E452DD03E550DD03E44EDD1E
:100F700020920E0120920F01F8940AB50B7F0ABD52
:100F8000789408952092130100914A010E7F0093F6
:100F90004A0100915E010E7F00935E0100914501C0
:100FA0000E7F00934501009159010E7F0093590176
:100FB00000910E0110910F010451120900931001CC
:100FC0001093110120920E0120920F0103E0009373
:100FD000170120921F012092280120922E010E94C9
:100FE000111200683FDE10E386DD0AB501FFEFDB7A
:100FF0000AB501FFAFDEE1DBF3980BB504600BBD72
:101000000895009112010F730E3158F0F298729802
:1010100000911201007C21F020920C0120920D0120
:101020000895F09B08950A3078F0F1990064F19BDF
:1010300000680093120106FF32C0F39930C020927D
:101040000E0120920F012BC000910C0110910D0197
:101050000030120521F1F2990895729A08EC00937C
:10106000E40063E0759AF19B0DC0009112010F77C7
:10107000009312016F987798000000006E9A769A9C
:10108000F29A0895009112010F7B009312016E985D
:101090007698000000006F9A779AF29A0895F09B74
:1010A00008956E9876986F987798F098F39B0895C6
:1010B00000911301013091F409E410E1A7DC0EE482
:1010C000A5DC03E5A3DC04E5A1DC0FE310E29EDC74
:1010D0000FE49CDC0BE49ADC0FE398DC0091130135
:1010E000039500931301089503B10095017F0295C4
:1010F000087106950695069510910A01102B110F9F
:10110000110F1C7310930A01143071F0183361F041
:10111000183089F0143379F000910B01007C00380D
:1011200089F00034C1F0089500910B010F7300683D
:1011300000930B01089500910B010F73006400935D
:101140000B0108951C3119F0103209F0089503E0E5
:1011500000930B0108951C3219F0103109F0089525
:1011600002E000930B01089500910B0101FD45C0C1
:10117000F49B0895F49800910801013019F00430AF
:10118000B9F10895F6990BC0F69A20922D0120929C
:101190002C0134DD49DD86DB00E07CD0089503E5D9
:1011A00010E134DC04E532DC0FE430DC02E52EDC57
:1011B00003E510E22BDC04E529DC0FE427DC02E583
:1011C00025DC8BD8A4D801E000931F0103E0009335
:1011D0002E0100911E01006845DD10E38CDC0BB58B
:1011E00004600BBD0AB501FFF2DAF698F79808958E
:1011F000F69B089503E04ED008950D7F00930B01F8
:1012000000FD0FC0F6990AC033D000910001109183
:1012100001010093020110930301089501E03AD007
:101220000895F6990AC00CD00091000110910101B7
:101230000093020110930301089502E02BD008955A
:10124000009123011091240181E00C32180749F02C
:1012500085E0080F121D0093230110932401809351
:101260001F010AE0009317010BB504600BBD089540
:10127000009123011091240180E00832180789F3BE
:1012800005501209009323011093240185E08093F7
:101290001F01E7CF64E1F799B9C0003051F0013088
:1012A00029F0023021F0033019F0089555C07AC0BA
:1012B00098C04427E4EDF4E290912D0180912C0137
:1012C000159105910817190711F400279FC01F3FBA
:1012D00011F04395F5CF00912C01003071F10F70A2
:1012E00099F410E100912C01003141F0F59B04C00C
:1012F000010F39F4010F05C0011B19F420922C01D4
:10130000089500932C01D5CF00912C010F7001306E
:1013100049F0F59B05C003950F7039F4039505C09E
:101320000A9519F420922C01089510912C01107F38
:101330000F70102B10932C01BCCF00912D010F3F8B
:1013400029F020922D0120922C01B3CF0AE00093C6
:101350002D0120922C01ADCFF59800912C01007F3A
:10136000D9F000912C010F7071F000912C010A95B9
:101370000F7009F40A9510912C01107F0F70102B3B
:1013800010932C0196CF00912C0110E1011B09F460
:10139000011B00932C018DCF00912D010A95009324
:1013A0002D0187CFF59A00912C01007FA1F00091CB
:1013B0002C010F7039F000912C0103950F70D9F6B4
:1013C0000395D9CF00912C0110E1010F09F4010F11
:1013D00000932C016ECF00912D01039500932D01F8
:1013E00068CF00912C01007F29F000912C010F7033
:1013F00039F0089500912C01005F00932C0159CF22
:1014000000912C010F5F00932C0153CFEBE0FAE029
:10141000E40FF21D099490C099C0ABC0B8C0CAC017
:10142000D1C0DAC096C120C224C21EC222C21CC2D0
:1014300020C21AC223C2E8C08CC116C21AC214C28A
:1014400018C212C216C210C219C2EDC082C10CC2AB
:1014500010C20AC20EC208C20CC206C20FC2F2C03B
:1014600078C102C206C200C204C2FEC102C2FCC1EF
:1014700005C2F7C06EC1F8C1FCC1F6C1FAC1F4C122
:10148000F8C1F2C1FBC1FCC064C1EEC1F2C1ECC144
:10149000F0C1EAC1EEC1E8C1F1C101C15AC1E4C164
:1014A000E8C1E2C1E6C1E0C1E4C1DEC1E7C106C1F5
:1014B00050C1DAC1DEC1D8C1DCC1D6C1DAC1D4C1E4
:1014C000DDC113C146C1D0C1D4C1CEC1D2C1CCC1CE
:1014D000D0C1CAC1D3C122C13CC1C6C1CAC1C4C1E5
:1014E000C8C1C2C1C6C1C0C1C9C1CDC1D6C10FC268
:1014F00047C285C292C2CBC208C348C380C3BBC324
:10150000C8C3F1C3D4C3EFC3E0C3EDC3FFC30CC46E
:1015100026C433C436C443C442C441C44EC45BC4AD
:1015200075C47CC496C49EC4ABC4B8C4C5C4E2C46C
:1015300000C520C540C55EC50DE410E367DA0FE4C1
:1015400065DA04E463DA05E461DA08950DE410E194
:101550005DDA01E45BDA0EE459DA05E557DA0FE308
:1015600010E254DA0FE352DA0FE350DA0FE34EDA07
:101570000895F8940AB502600ABD78941ED91DDB5F
:1015800050E00BB502600BBD8DD9EFDB08CE01E456
:1015900010E13CDA05E53ADA04E538DA0FE436DA48
:1015A0000FE310E233DA0FE331DA0FE32FDA0FE360
:1015B0002DDA0895F8940AB50D7F0ABD7894FDD808
:1015C000C9DBEDCD00E510E321DA02E51FDA0FE417
:1015D0001DDA07E41BDA089504E510E117DA01E4E7
:1015E00015DA07E413DA01E311DA0FE310E20EDA99
:1015F0000FE30CDA0FE30ADA0FE308DA00E832DB74
:1016000010E179DA4FD9089504E510E1FFD901E43A
:10161000FDD907E4FBD902E3F9D901E823DB10E1A6
:101620006ADA40D9089504E510E1F0D901E4EED971
:1016300007E4ECD903E3EAD902E814DB10E15BDA52
:1016400031D9089504E510E1E1D901E4DFD907E4D7
:10165000DDD904E3DBD903E805DB10E14CDA22D95C
:10166000089504E510E1D2D901E4D0D907E4CED938
:1016700005E3CCD904E8F6DA10E13DDA13D9089590
:1016800004E510E1C3D901E4C1D907E4BFD906E3F9
:10169000BDD905E8E7DA10E12EDA04D9089504E5AA
:1016A00010E1B4D901E4B2D907E4B0D907E3AED967
:1016B00006E8D8DA10E11FDAF5D8089504E510E15C
:1016C000A5D901E3A3D90AE3A1D905E39FD900E88D
:1016D000C9DA10E110DA01E80EDA02E80CDA03E800
:1016E0000ADA04E808DADED8089504E510E18ED9B4
:1016F00001E38CD90AE38AD906E388D900E8B2DA93
:1017000010E1F9D901E8F7D902E8F5D903E8F3D9EE
:1017100004E8F1D905E8EFD9C5D8089504E510E14A
:1017200075D901E373D90AE371D907E36FD900E8EA
:1017300099DA10E1E0D901E8DED902E8DCD903E862
:10174000DAD904E8D8D905E8D6D906E8D4D9AAD890
:101750000895F79A0F9373DAB0DAA4DAB9DA43DAB4
:10176000A7E6B1E000912C010151102F0F70107FFE
:10177000129589E0189FA00DB11DA0933001B09380
:101780003101A00FB21D1C910F91013031F00230D8
:1017900049F0033009F00AC039C01A951E3F31F4F0
:1017A0001FE804C01395103909F41FEF1C931F3F65
:1017B000D1F0012F0E94A8020E2D003309F40FE38F
:1017C00010E124D90D2D22D90C2D20D900E31ED9EA
:1017D00010E20FE31BD90FE319D90FE317D90FE379
:1017E00015D929D808950AE310E110D90AE30ED9D2
:1017F0000AE30CD90AE30AD910E20FE307D90FE391
:1018000005D90FE303D90FE301D90895F7D9F79864
:1018100000912C010170B1F40E910F3F99F41196D3
:101820000D910F3F79F400912C010F7008501FEFBC
:101830001D930395E9F700912C01007F085F009349
:101840002C01DECD00912C010F70093009F0D8CDAC
:1018500000912C01007F003808F0EDD300912C019D
:10186000007F00932C01C6CDF79A0F9310DA3BDA74
:1018700076CFF79A0F9316DA2BDA71CFF79A0F9388
:1018800011DA3CDA6CCF04E510E3C0D805E4BED829
:101890000DE4BCD800E5BAD80895F79AA0913701B5
:1018A000B0913801013029F0023051F0033069F174
:1018B0000EC01597A832B20550F4A8E2BB2707C0A6
:1018C000159681E0AE35B80710F0AEE5B1E0A09313
:1018D0003701B09338018D010E9475020E2D10E181
:1018E00095D897D90D2D92D80C2D90D800E48ED88C
:1018F00010E20FE38BD80FE389D80FE387D80FE30B
:1019000085D8D0D9DAD9E4D90895F79873CDF79A64
:10191000A0913901B0913A01013029F0023051F023
:10192000033061F10EC01597A832B20550F4A8E259
:10193000BB2707C0159681E0AE35B80710F0AEE5BD
:10194000B1E0A0933901B0933A018D010E94750274
:101950000E2D10E15BD85DD90D2D58D80C2D56D821
:1019600000E454D810E20FE351D80FE34FD80FE34F
:101970004DD80FE34BD88BD9B6D90895F7983ACD07
:10198000F79AA0913B01B0913C01013029F002305F
:1019900051F0033061F10EC01597A832B20550F432
:1019A000A8E2BB2707C0159681E0AE35B80710F056
:1019B000AEE5B1E0A0933B01B0933C018D010E94E4
:1019C00075020E2D10E122D824D90D2D1FD80C2D13
:1019D0001DD800E41BD810E20FE318D80FE316D887
:1019E0000FE314D80FE312D85DD988D90895F7987A
:1019F00020922C014CD956D960D916D95ACC0AE577
:101A000010E30E94060505E40E94060509E40E9411
:101A1000060504E50E9406050895F79A10911D0138
:101A2000013029F0023041F0033079F109C01A95F4
:101A30001F3F31F413E604C01395143609F411273F
:101A400010931D01012F0E94950202E310E10E94F4
:101A5000060500E30E9406050D2D0E9406050C2DCB
:101A60000E94060510E20FE30E9406050FE30E94A4
:101A700006050FE30E9406050FE30E940605D1D478
:101A80000068F0D810E337D80895F798B3CCF79AE8
:101A900010911C01013029F0023041F0033099F11E
:101AA00009C01A951F3F31F41BE004C013951C3088
:101AB00009F4112710931C0100911B0103950E944A
:101AC00095020D2D10E30E9406050C2D0E940605BF
:101AD000A0D80FE312E20E9406050FE30E9406055C
:101AE00000911C0103950E9495020D2D12E10E94A8
:101AF00006050C2D0E94060594D40068B3D810E3A7
:101B00000E947B050895F79875CCF79A80911B0188
:101B1000013029F0023051F00330A9F10CC0A9D4F2
:101B20008A958F3F41F4812F8A9505C0A2D4839571
:101B3000811709F4882780931B0100911B010395ED
:101B40000E9495020D2D10E10E9406050C2D0E94A9
:101B500006050FE310E20E9406050FE30E9406054A
:101B600000911C0103950E9495020D2D12E30E9425
:101B700006050C2D0E94060554D4006873D810E3A6
:101B80000E947B050895F7984FD834CCF79A1091AE
:101B90001A01013029F0023041F0033071F109C01F
:101BA0001A951F3F31F417E104C01395183109F459
:101BB000112710931A01012F0E9495020D2D003359
:101BC00009F40FE310E10E9406050C2D0E940605A2
:101BD0000FE310E20E9406050FE30E9406050E9433
:101BE000F305009119010E9495020D2D12E30E9448
:101BF00006050C2D0E9406050895F798FBCBF79A71
:101C000010911901013029F0023041F0033069F1DF
:101C100009C01A951F3F31F41BE304C013951C3310
:101C200009F411271093190100911A010E949502DD
:101C30000D2D003309F40FE310E30E9406050C2D6F
:101C40000E940605009119010E9495020D2D12E1D6
:101C50000E9406050C2D0E9406050FE312E20E9469
:101C600006050FE30E9406050895F79820922C01BF
:101C70000E94FE051ECB06E410E30E94060505E463
:101C80000E9406050EE40E94060503E50E94060573
:101C9000089508E410E30E9406050FE40E9406057B
:101CA00003E40E94060508E40E94060508950DE479
:101CB00010E30E94060509E40E94060504E50E945F
:101CC000060504E50E94060508950EE410E30E944F
:101CD000060509E40E94060505E40E94060504E4E1
:101CE0000E940605089500912C010F700E94950234
:101CF0000C2D10E30E94060500E30E9406050FE389
:101D00000E9406050DE40E940605089502E510E311
:101D10000E94060505E40E94060503E50E940605EB
:101D20000FE30E94060508950FE310E10E940605E7
:101D30000FE40E9406050BE40E9406050FE30E94D3
:101D400006050FE310E20E9406050FE30E94060558
:101D50000FE30E9406050FE30E940605089501E4C3
:101D600010E30E94060504E40E94060501E40E94B7
:101D7000060500E50E94060508950E94A101F69857
:101D8000089505E510E30E94060502E50E94060598
:101D90000CE40E94060501E40E940605089504E48F
:101DA00010E30E94060501E40E94060504E50E9476
:101DB000060505E40E940605089506E510E30E9465
:101DC000060505E40E9406050EE40E94060504E5EA
:101DD0000E94060508950EE410E30E9406050FE434
:101DE0000E94060502E50E9406050DE40E94060514
:101DF0000FE310E20E9406050FE30E9406050FE3C1
:101E00000E9406050FE30E94060508950BB5077FA3
:101E10000BBD0E9452040E94B506C1C909E410E33B
:101E20000E9406050EE40E94060506E50E940605CE
:101E300005E40E9406050FE310E20E9406050FE389
:101E40000E9406050FE30E9406050FE30E940605A7
:101E500008950BB508600BBD0E9452040E94B506A0
:101E60009EC908950FE410E30E94060506E40E944F
:101E7000060506E40E94060503E50E94060508958E
:101E80000BE210E30E94060500E30E94060500E451
:101E90000E9406050FE30E940605089504E410E37E
:101EA0000E94060502E40E94060505E50E9406055B
:101EB00007E40E940605089506E410E10E94060565
:101EC00009E40E94060502E50E9406050DE40E9451
:101ED000060505E00E94950206E510E20E9406054F
:101EE0000E2D0E9406050D2D0E9406050C2D0E9448
:101EF0000605089506E410E10E94060505E50E9426
:101F000006050AE50E9406050AE50E9406050091FD
:101F100032010E9495020FE310E20E9406050FE3D2
:101F20000E9406050D2D0E9406050C2D0E94060537
:101F3000089500E510E10E9406050FE40E940605E1
:101F400003E50E94060509E40E94060500910E01C2
:101F500010910F010E9475020F2D10E20E940605DC
:101F60000E2D0E9406050D2D0E9406050C2D0E94C7
:101F70000605089506E510E10E94060504E50E94A5
:101F800006050FE40E94060500E50E940605009183
:101F90001001109111010E9475020F2D10E20E9494
:101FA00006050E2D0E9406050D2D0E9406050C2D1E
:101FB0000E940605089502E510E10E94060507E566
:101FC0000E94060501E40E94060509E50E94060537
:101FD000009127010E9495020FE310E20E9406057E
:101FE0000E2D0E9406050D2D0E9406050C2D0E9447
:101FF0000605089506E510E10E94060502E40E9428
:10200000060501E40E94060504E50E94060500910C
:102010003301109134010E9475020F2D10E20E94CD
:1020200006050E2D0E9406050D2D0E9406050C2D9D
:102030000E9406050895003829F0003939F0003A69
:1020400049F0089585E0A6EAB1E007C086E0AFEA6E
:10205000B1E003C087E0A8EBB1E0C7E6D1E019E04A
:102060000D9109931A95E1F719978A95C1F708958B
:102070003FB60F931F9300912B01039500932B0103
:10208000033040F011F0063050F06F9877986E985A
:10209000769809C06E9876986F9A779A04C06F9870
:1020A00077986E9A769A0F3088F020922B010091E3
:1020B000290110912A01011720F4039500932901A9
:1020C00005C000916E000D7F00936E001F910F916F
:1020D0003FBE1895609928C0F29B189563E03FB603
:1020E000AF93BF93619917C0F39B09C0A0910E01F4
:1020F000B0910F011196A0930E01B0930F01A09122
:102100000C01B0910D01A030B20529F01197A093F8
:102110000C01B0930D01A0911201A07CA0931201BB
:10212000BF91AF913FBE18952F9828980E945701F4
:102130000E946F040FE410E30E94060506E40E946B
:10214000060506E40E9406050FE30E9406050E94AC
:10215000650507E003BF8895FFCF3FB60F931F9338
:1021600008EC0093E40063E00E9474081F910F9153
:102170003FBE18953FB60F931F9303B10095017FA3
:1021800002950770003079F0109109010093090160
:1021900001130CC03F3F51F03395353039F40093B3
:1021A0000801F49A03C0332720920901009112011B
:1021B0000F730F3329F00091120103950093120160
:1021C0001F910F913FBE18953FB60F931F938F93AA
:1021D00000912E010395037000932E0179F4009174
:1021E000280103950093280100911F01002331F07D
:1021F0000A9500931F0111F42092280100912201F9
:102200007394701609F021C0772404E00093220132
:10221000F8940AB500680ABD7894F3990EC000914D
:1022200017010A950093170141F404EB009317017D
:10223000F8940AB500610ABD7894603031F06A956F
:1022400021F400EC0093E40075988F911F910F9199
:102250003FBE18950EE500937C00000000000000D2
:1022600004EC00937A0000917A0006FDFCCF04E0B4
:1022700000937A0000917800109179000093330167
:102280001093340182E00231180768F009E810E188
:102290000E948005009133011091340182E00033E7
:1022A000180708F041CF0895F39B089502E40093C6
:1022B0007C0000000000000004EC00937A00009114
:1022C0007A0006FDFCCF04E000937A0000917800CC
:1022D000109179008FEF93E0801B910B8093140194
:1022E00008950AB507FF0895F8940AB50F770ABD57
:1022F0007894009118010395009318010C3309F0AC
:1023000082C02092180100911901039500931901D0
:10231000009119010C3309F076C020921901009147
:102320001A01039500931A0100911E01043049F42B
:1023300000911A010B3029F4F8940AB504600ABD23
:1023400078940AB503FD23C000911B010831F8F011
:1023500000911E010630D9F400911C01093019F0DA
:10236000023049F014C000911A01033081F40A953B
:1023700000931A0107C000911A01023041F403953D
:1023800000931A01F8940AB508600ABD7894009188
:102390001A01083109F037C0F8940AB5077F0ABD61
:1023A000789420921A0100911B01039500931B0160
:1023B00000911E01039500931E01073019F40027B8
:1023C00000931E0100680E94320610E30E947B0504
:1023D0000AB501FF0E94E7034CD000911B010117D1
:1023E00091F420921B0100911C01039500931C01A4
:1023F00000911C010C3039F420921C0100911D0148
:10240000039500931D010AB502FF0AC0F39908C0A5
:102410000E94FE050E9414060E9452040E94A1011F
:10242000089500911C01E2E9F4E2E00FF21DC09072
:102430001B01C394D490E0901D0100911C01023057
:1024400008F4EA94CD0CCE0CE694E69404E10695EB
:102450000695CE0CC00E04E6C00E07E0C01610F0C4
:10246000C01AFCCF0C2D015008F406E000931E01A9
:10247000089500911C01EEE9F4E2E00F149100913F
:102480001D01037029F400911C01013009F413951A
:1024900008951C1F0205070A0C0F121417191F1CA0
:1024A0001F1E1F1E1F1F1E1F1E1F2A85C666D84FF8
:1024B000803E423110272D1F081936146A10670D0F
:1024C000000B1209850743063C056604B503240387
:1024D000AC020000000000100011002000210100EB
:1024E0000110011101120113011401150116011748
:1024F00001180119012001210122012301240125D4
:10250000012601270128012901300131013201335F
:1025100001340135013601370138013901400141EB
:102520000142014301440145014601470148014977
:1025300001500151015201530154015501560157F7
:102540000158015901600161016201630164016583
:10255000016601670168016901700171017201730F
:10256000017401750176017701780179018001819B
:102570000182018301840185018601870188018927
:1025800001900191019201930194019501960197A7
:102590000198019901A001A101A201A301A401A533
:1025A00001A601A701A801A9020002100220023021
:1025B0000300031003200330034003500400041001
:1025C0000411042004210430043105000510060024
:1025D0000610070007100720073008000810081130
:1025E00008200821090009100A000A100A200A30F0
:0825F0000A400A500A60FFFFD7
:00000001FF
